:1000000009298030A100FE30A7200130A7207530DB
:10001000A7003030BE28A101A117AF00AF08031D13
:100020001328030114280130AF020310A20CA20C04
:10003000A20CC0302205403EAF07FE30A7202F089B
:10004000A728A101A117AF00FE30A7202F08A728DD
:10005000A401AA00AB01A01124080319A0150530C2
:10006000A3002730A900103041200330A900E83058
:100070004120A90164304120A9010A3041202A0809
:100080004828A8002B08A7002A08A600D220260886
:10009000A600A3030319A011240803195228230260
:1000A000031859282608031DA011A0195928303E0D
:1000B000A7280800AD0006118611831606118611C7
:1000C0000F30860583122D08A01884283E30A70023
:1000D0008030BE203330AC0098201330A700883029
:1000E000BE2098206430BD2098206430BD2022308E
:1000F000AC009820283083200C30832006308320E9
:10010000A0142D0884282014AC00201C92288611ED
:10011000033C031C972897200530A700DC30BE2045
:10012000031408002014FE3C0319A5288615201C82
:10013000201006150F3086052C08F03986040611AC
:10014000AC0E201898283230BD202D080429A11BA0
:100150005A2883178001840AFF3E031DAA28042918
:10016000A901A800FF30A807031CA907031C042944
:100170000330A700DF30BE20B228A701E83EA6006A
:10018000A709FC30031CC728A6070318C428A60724
:100190000000A70FC4282618CD28A61CD1280000CF
:1001A000D1280800AB01AA011030AC00270DAA0D20
:1001B000AB0D2808AA022908031C290FAB0203185B
:1001C000E8282808AA0729080318290FAB070310F5
:1001D000A60DA70DAC0BD628260804291030B000B8
:1001E000A701A601AD0CAC0C031CFC282808A6072F
:1001F00029080318290FA707A70CA60CAB0CAA0CFB
:10020000B00BF2282A080429831383120313000079
:100210000800A00107309F00E03083168500FF3002
:1002200086008113831285018601203084006030AE
:10023000AA20A03084005030AA2020308400303022
:10024000A920C830B020012077305A205A205A20E7
:100250002E305A2070305A2069305A2063305A208C
:1002600062305A2061305A2073305A2069305A2047
:1002700063305A202E305A206E305A206C305A206B
:100280000B30A900B830B120012044305A2043304F
:100290005A2046305A2032305A2034305A204E30BC
:1002A0005A204C305A2042305A2020305A205A20AE
:1002B00056305A202D305A2032305A200730A900AB
:1002C000D030B12001204C305A2044305A205230D6
:1002D0005A2020305A2061305A2066305A2072301D
:1002E0005A2065305A2067305A2065305A206C30C9
:1002F0005A2065305A206E305A2086188529851F6D
:1003000083290514842905107D29012053305A20A2
:1003100069305A2067305A206E305A2061305A2096
:100320005A206C305A2020305A207A305A206F30B0
:100330005A2065305A206B305A2065305A206E3072
:100340005A2036140512831605128312342AC3016B
:100350003C03A500C90149082502031CC029E3216B
:10036000B61CBE294308A6004908A200A601A20A9D
:100370000314A60DA20BB9292608C304C90FAB2983
:10038000B2014308B100B20CB10CB20CB10CB20C0A
:10039000B10CB20CB10C0F30B2053208AD0031080F
:1003A000AC00A9010A30A800EE20B1002B08B20071
:1003B000B4014308B3000F30B3050030B405310871
:1003C0003307C3000800BA01B9010618F829013043
:1003D000B020B90A0319BA0A0B303A02031CF729F4
:1003E000031DF629B9303902031CF729C62CE5296B
:1003F0009B30B0200618B614061CB610361C142A02
:10040000AD014408AC00A9011830A800EE20B100ED
:100410002B08B2003208A7003108A600A9013A3023
:10042000A800D220BD00272A8030A1000130A20000
:100430003D080D200230A40044082920030136198C
:10044000013EB618013A03193611031D3615C40AC8
:1004500085140130A900F430B1208510A901F030D5
:10046000A8002808B1200800BB01C4013612361AC2
:10047000D12ABA01B901061C4E2AB90A0319BA0ACF
:100480000130B020AF303A02031C4D2A031D4C2A24
:10049000C9303902031C4D2AC62C3B2ABA01B901C6
:1004A00006188A2AB90A0319BA0A0A30B02036187F
:1004B0007E2A39080B3A3A04031D692A8030A100CC
:1004C0000130A2003D080D2035305A2039305A2025
:1004D0007D2A3908193A3A04031D702A85147D2AA9
:1004E00039084B3A3A04031D772A85107D2A3908CA
:1004F000FA3A3A04031D7D2AC62C892A11303A02A1
:10050000031C892A031D882A95303902031C892A75
:10051000C62C502A41303B02031C8F2AC62CBB0A32
:100520003A08031D972A65303902031C982A3616AB
:10053000361CD02AAD013B08AC00A9011830A80038
:10054000EE20B1002B08B2003208A7003108A60047
:10055000A9014130A800D220BD008030A100803028
:10056000212053305A2069305A2067305A206E308B
:100570005A2061305A205A206C305A2020305A209C
:1005800067305A2065305A2076305A206F305A2012
:100590006E305A2064305A2065305A206E305A200E
:1005A000372A361CF32A012049305A206E305A204F
:1005B00069305A2074305A2069305A2061305A20EC
:1005C0006C305A2069305A2073305A2065305A20D6
:1005D00072305A2065305A206E305A202E305A2000
:1005E0005A205A20622B0F30BD000130A2003D0876
:1005F0000B20A101B61D0B2B3B3041020318022B2F
:10060000C10A0A2BC101173045020318092BC50A7C
:100610000A2BC5010F2B4208C1004608C500051B67
:100620001F2B4508031D172B0C30C7001E2B0D3048
:100630004502031C1E2B0C304502C700242B450825
:10064000C70020305A205A200A30470203182A2BAC
:1006500020305A208030A100470828203A305A2004
:100660000230A400410829203A305A2030305A2064
:100670005A20051B4B2B0C3045020318442B6130CC
:100680005A206D305A20482B70305A206D305A2035
:100690001530BD004D2B1730BD0041080319013046
:1006A000031D0301B5001E30410203190130031D73
:1006B00003013504B5000130861803013504031920
:1006C000622B9E2C361E9C2CE3210130C9000F307A
:1006D000490203186E2BE321C90F672B3611B6119F
:1006E000E321E321E321B61C772B0514782B0510B9
:1006F0001230C900143049020318812BE321C90FBD
:100700007A2BE3210730BC00A7214308C200E32174
:10071000361D8B2BB6150630BC00A7214308C6003A
:10072000E321361D942BB6150630BC00A7214308E3
:10073000BE000330BC00A7214308C8000530BC0040
:10074000A7214308C0000830BC00A7214308BF0010
:10075000E321361DAC2BB615361CB22BB619B12BC6
:1007600036100120B6199B2C80302120A1010130C8
:100770004802031DC02B4D305A2061305A20F52B02
:1007800002304802031DC92B44305A2069305A20D8
:10079000F52B03304802031DD22B57305A206F30FF
:1007A0005A20F52B04304802031DDB2B44305A201D
:1007B0006F305A20F52B05304802031DE42B5630CC
:1007C0005A2072305A20F52B06304802031DED2BBB
:1007D0005A305A2061305A20F52B07304802031D49
:1007E000F52B5A305A206F305A208030A1008330C8
:1007F00021203E08282020305A2001304002031DCD
:10080000082C6A305A2061305A206E305A20802CD1
:1008100002304002031D132C66305A2065305A20E6
:1008200062305A20802C03304002031D1E2C6D3094
:100830005A2072305A2074305A20802C04304002E2
:10084000031D292C61305A2070305A2072305A20F2
:10085000802C05304002031D342C6D305A20653049
:100860005A2069305A20802C06304002031D3F2C4C
:100870006A305A2075305A206E305A20802C07304A
:100880004002031D4A2C6A305A2075305A206C30C1
:100890005A20802C08304002031D552C61305A200C
:1008A00075305A2067305A20802C09304002031DD1
:1008B000602C73305A2065305A2070305A20802CBA
:1008C0000A304002031D6B2C6F305A206B305A20C7
:1008D00074305A20802C0B304002031D762C6E3071
:1008E0005A206F305A2076305A20802C0C3040022B
:1008F000031D802C64305A2065305A2063305A2002
:10090000051B8F2C20305A2027305A208030A10020
:100910000230A4003F08292020305A209B2C203090
:100920005A2032305A2030305A208030A100023014
:10093000A4003F0829209D2CC62C342A851FA52CF5
:100940000512831605128312A72C8316051683122F
:100950009B30B020410803190130031D0301B5008D
:1009600001308618030135040319B72C05158515C8
:1009700085140130A900F430B120051185118510CE
:100980000130A9004A30B120C40A652B012047304C
:100990005A2065305A205A206E305A2020305A2072
:1009A00073305A2069305A2067305A206E305A20EE
:1009B00061305A205A206C305A2020308400603038
:1009C000AA20A03084005030AA202030840030308B
:1009D000A9200618B616061CB61203010618013E19
:1009E000B61A013C031DFA2CB70A0319B80A0130E4
:1009F000B020ED2C0301B61A0130013A0319B612EA
:100A0000031DB61603010618013EB61A013C031D6C
:100A10000F2DB70A0319B80A0130B020022D033098
:100A20003802DE30031937020318DD2C3614342A5D
:02400E00503F21
:00000001FF
